:10000000020A40120A3112005AD2AF7BFF7A0A79F3
:10001000561200F07F017E00120A1AD3E5279400E1
:100020007480948040EE1527E52770E8D3E5269488
:100030000074809480401EE4F508E508C3952650BE
:100040001474002508F582E43400F583E0FF120AF9
:100050004C050880E5E4F52680BA750940750A0369
:10006000750E00750DC2750C01750B007510017BC6
:10007000007A0079097F031208477D017F01120988
:0A0080007253BAFD22AE07020A4CCB
:10008B000209C7E518240CF8E60518227809300791
:10009B0002780CE475F0011208110206612000EBE6
:1000AB007F2ED2008018EF540F2490D43440D4FF0D
:1000BB0030040BEF24BFB41A0050032461FFE51981
:1000CB0060021519051CE51C7002051B30070D7825
:1000DB0009E475F001120811EF0207C902008574DB
:1000EB0003D2078003E4C207F5188B098A0A890B30
:1000FB00E4F519F51BF51CE51960077F201200C903
:10010B0080F5751AFFC201C200C202C203C205C24A
:10011B0006C208120097FF700D3007057F00120012
:10012B00DAAF1CAE1B22B4255FC2D5C204120097F6
:10013B00FF24D0B40A00501A75F00A781930D5058F
:10014B0008B6FF0106C6A426F620D5047002D2031A
:10015B0080D924CFB41A00EF5004C2E5D2040202B6
:10016B00DAD20180C6D20080C0D20280BCD2D58048
:10017B00BAD20580B47F201200C92002077401B5E2
:10018B00190040F112008EFF1200C9020102D208C1
:10019B00D206809512008EFB12008EFA12008EF999
:1001AB004A4B700679AB7A037BFF20022EE5196070
:1001BB002A7E008E8275830012067A60060EEE652B
:1001CB001A70F0C2D5EBC0E0EAC0E0E9C0E0EE1275
:1001DB000321D0E0F9D0E0FAD0E0FB120661FF601A
:1001EB00AAEBC0E0EAC0E0E9C0E01200C9D0E0240D
:1001FB0001F9D0E03400FAD0E0FBE51A0460DCD55D
:10020B001AD980877BFF7A03791DD202809C7910E3
:10021B0080027908C206C2088008D2D5790A800408
:10022B00790AC2D5E51A047002F51AE4FAFDFEFF4D
:10023B0012008EFC7B0820011312008EFD7B103008
:10024B00000A12008EFE12008EFF7B20EC3382D54B
:10025B0092D55013C3E43000069FFFE49EFEE420CA
:10026B0001039DFDE49CFCE4CBF8C201EC700CCFC8
:10027B00CECDCCE824F8F870F38017C3EF33FFEE44
:10028B0033FEED33FDEC33FCEB33FB994002FB0FFC
:10029B00D8E9EB300105F8D0E0C448B201C0E00A60
:1002AB00EC4D4E4F78207B0070C2EAB51A0040BC73
:1002BB00C0E0120323D0F0D0E0200104C4C0E0C49E
:1002CB00B201C0F01200B2D0F0D5F0EB0201021275
:1002DB000821019F5302195801704C016C42021DF9
:1002EB004F022544022549018543022B55020F4637
:1002FB00020F45020F4703CB5001742D01782E01DD
:10030B009B2B017C2301992003B42A013448000064
:10031B0001933F3F3F00790AA2D520031430050912
:10032B00B910020404B9080104A2D5200602500139
:10033B00042002689202B519005034C0E07F2030CF
:10034B0003197F30A20272067205500F12037AC294
:10035B0002C206C205C2087F30800F300503E9C018
:10036B00E01200C9300503D0E0F9D0E0B519CC306C
:10037B0005177F30B9100C1200C97F583004077F66
:10038B00788003B908031200C93002057F2D0200E3
:10039B00C97F202008F87F2B2006F322920280CF02
:1003AB00286E756C6C2900D20112008E3001F8C2D8
:1003BB0001781930D50108F60201342D5043495804
:1003CB0012008E2403B405004001E49003C693127F
:1003DB0000BA743A1200BAD203751904020219EF6B
:1003EB00D394077480948040037FFF22120661FE32
:1003FB00D394037480948040037FFF22EF7044EE0C
:10040B00700B90000112067AF4529352941206610B
:10041B006401700B90000112067A4293F45294120D
:10042B000661FE6402700A90000112067A42934242
:10043B0094EE6403700D90000112067AFEF4529351
:10044B00EE4294EF64017046120661FE700B900051
:10045B000112067AF452915292EE6401700B9000E5
:10046B000112067A4291F452921206616402700AEA
:10047B0090000112067A4291429212066164037057
:10048B000D90000112067AFEF45291EE4292EF6447
:10049B00027046120661FE700B90000112067AF490
:1004AB0052955296EE6401700B90000112067A423F
:1004BB0095F452961206616402700A9000011206BE
:1004CB007A429542961206616403700D90000112F8
:1004DB00067AFEF45295EE4296EF640370461206CE
:1004EB0061FE700B90000112067AF452B152B2EE1B
:1004FB006401700B90000112067A42B1F452B212F1
:10050B0006616402700A90000112067A42B142B28F
:10051B001206616403700D90000112067AFEF4520C
:10052B00B1EE42B2EF64047046120661FE700B909E
:10053B00000112067AF452B352B4EE6401700B90C0
:10054B00000112067A42B3F452B4120661640270CF
:10055B000A90000112067A42B342B4120661640398
:10056B00700D90000112067AFEF452B3EE42B4EF16
:10057B0064057046120661FE700B90000112067A3C
:10058B00F452C952CAEE6401700B90000112067A44
:10059B0042C9F452CA1206616402700A9000011239
:1005AB00067A42C942CA1206616403700D900001BB
:1005BB0012067AFEF452C9EE42CAEF640670461276
:1005CB000661FE700B90000112067AF452CB52CCEE
:1005DB00EE6401700B90000112067A42CBF452CC00
:1005EB001206616402700A90000112067A42CB4235
:1005FB00CC1206616403700D90000112067AFEF4B2
:10060B0052CBEE42CCEF64077049120661FF7E00BD
:10061B00700B90000112067AF452E152E2EF640182
:10062B004E700B90000112067A42E1F452E2120670
:10063B00616402700A90000112067A42E142E212F2
:10064B0006616403700D90000112067AFFF452E10B
:10065B00EF42E27F0022BB010689828A83E02250AF
:10066B0002E722BBFE02E32289828A83E49322BB48
:10067B00010CE58229F582E5833AF583E0225006E9
:10068B00E92582F8E622BBFE06E92582F8E222E59F
:10069B008229F582E5833AF583E4932275F0087598
:1006AB008200EF2FFFEE33FECD33CDCC33CCC582A2
:1006BB0033C5829BED9AEC99E58298400CF582EE5E
:1006CB009BFEED9AFDEC99FC0FD5F0D6E4CEFBE446
:1006DB00CDFAE4CCF9A88222B800C1B90059BA000E
:1006EB002DEC8BF084CFCECDFCE5F0CBF97818EF69
:1006FB002FFFEE33FEED33FDEC33FCEB33FB10D76A
:10070B0003994004EB99FB0FD8E5E4F9FA2278182A
:10071B00EF2FFFEE33FEED33FDEC33FCC933C91085
:10072B00D7059BE99A4007EC9BFCE99AF90FD8E0B7
:10073B00E4C9FAE4CCFB2275F010EF2FFFEE33FE89
:10074B00ED33FDCC33CCC833C810D7079BEC9AE8FC
:10075B0099400AED9BFDEC9AFCE899F80FD5F0DA7D
:10076B00E4CDFBE4CCFAE4C8F922EB9FF5F0EA9E6A
:10077B0042F0E99D42F0E89C45F022E8600FECC3A3
:10078B0013FCED13FDEE13FEEF13FFD8F122BB01AB
:10079B000DE58229F582E5833AF5830207E85007D8
:1007AB00E92582F80207DBBBFE07E92582F8020781
:1007BB00F4E58229F582E5833AF583020801BB0152
:1007CB000689828A83F0225002F722BBFE01F322B4
:1007DB00E6FB08E6F908E6FA08E6CBF822E0F8A310
:1007EB00E0F9A3E0FAA3E0FB22E2FB08E2F908E25E
:1007FB00FA08E2CBF822E493F8740193F9740293AC
:10080B00FA740393FB22FAE6FB0808E6F925F0F6E7
:10081B0018E6CA3AF622D083D082F8E493701274A9
:10082B000193700DA3A393F8740193F5828883E46D
:10083B00737402936860EFA3A3A380DF8B128A13F8
:10084B008914EF6403600302096F752203F523F526
:10085B0024F525F526F527F528FFEFC394207480A2
:10086B009480500F74202FF582E43400F583E4F06C
:10087B000F80E7E4FFEFC3942074809480500F74D3
:10088B00002FF582E43400F583E4F00F80E7AB1220
:10089B00AA13A914120661FF7E0064C06008EF64FE
:1008AB00406003020958EF64C04E700543AC808072
:1008BB000353AC7F9000021207997F007E607D543A
:1008CB007C001206E38F188E178D168C15E4FFFE35
:1008DB007D01FCAB18AA17A916A815C31207754002
:1008EB00037FFF22C3E49518F518E49517F51774E9
:1008FB00019516F516E49515F515AB12AA13A91467
:10090B0090000112067A64027026538EEF53ACBF2F
:10091B00538EF7438E04AF18AE17AD16AC1578088F
:10092B001207868FD68518D753AFFB438E108020C6
:10093B0043AC40AF18AE17AD16AC1578081207864E
:10094B008FD48518D553D1F043D10A80037FFF2272
:10095B0090000712067AC454F0FFE5AC54EF4FF544
:10096B00AC7F00227FFF22EFD394017480948050E0
:10097B000EEF33333354F8FFE5AF54F74FF5AFEDCC
:10098B00FF7E00D3940374809480502DEF70065338
:10099B00EEFE53DFFEEF64014E700653EEFE43DFB7
:1009AB0001EF64024E700643EE0153DFFEEF64036A
:1009BB004E700643EE0143DF017F0022C0E0C0838F
:1009CB00C082C0D075D000C007E5AC54016029537C
:1009DB00ACFEE5287022C3E52694207480948040F9
:1009EB0003752600AF26052674002FF582E434002C
:1009FB00F583E5ADF0752705E5AC5402600653AC05
:100A0B00FD752500D007D0D0D082D083D0E0327DC9
:100A1B00A37C08ED1D70011C144C70F7EF1F7001C7
:100A2B001E144E70EA22750A03E4F509FB7A00796D
:100A3B0009FF0203EA787FE4F6D8FD7581280200EE
:100A4B00038FAD752501E52570FC225354433820E7
:100A5B00554152543320546573742050726F677232
:080A6B00616D6D65210D0A00AB
:00000001FF
